:100000001DC037C036C035C034C033C032C031C067
:1000100030C02FC02EC02DC02CC02BC02AC029C07C
:1000200028C027C026C025C024C023C022C021C0AC
:1000300020C01FC01EC01DC01CC01BC011241FBE7D
:10004000CFEFD1E0DEBFCDBF11E0A0E0B1E0ECE644
:10005000F1E002C005900D92AE30B107D9F721E072
:10006000AEE0B1E001C01D92A431B207E1F752D079
:100070007BC0C6CF0F931F9300E010E098010617D6
:1000800017072807390759F0E7E8F3E13197F1F747
:1000900000C000000F5F1F4F2F4F3F4FF0CF1F9149
:1000A0000F91089586B197B1813022E0920714F044
:1000B00080E090E008958093B0008091B10087FFC8
:1000C000FCCF0895F8DF80E090E008958A3010F4C6
:1000D000805D01C0895CEFCFCF93C82F82958F7070
:1000E000F5DF8C2F8F70CF91F1CFCF93C82F892F51
:1000F000F3DF8C2FCF91F0CF8AB38F7A8ABBD59A5A
:1001000080E48093B20080E091E0909311018093AD
:1001100010010895F1DF80EF8093740080E189B9C8
:1001200082E288B914B884EE85B983E080936000D8
:1001300000E010E0C0E0D0E00032110554F4B2DF7E
:10014000C80FD91F82E48A95F1F700C00F5F1F4FD7
:10015000F3CF80E0B0DFCE01969587959695879591
:0C016000C4DF8AE0A8DFE4CFF894FFCFF2
:0E016C00000000020000000062000000000021
:00000001FF
